:100276007B017D807F021201CEE4FF120424E47527
:100286000F80750E25F50DF50CF510751110FF7E16
:10029600247DF4FC12022D7F941204387F02120290
:0B02A600B1EF60F87F0212031180EC42
:10037F00E4F59AF591F5A1F59BF592F5A2F5A0F5A7
:04038F0090F5802243
:1001CE00EF701CEB7006EDF4529A529BBB0107EDDB
:1001DE00F4529AED429BEB64027043ED429A22EF89
:1001EE006401701CEB7006EDF452915292BB010744
:1001FE00EDF45291ED4292EB64027022ED429122A7
:10020E00EF64027019EB7006EDF452A152A2BB011D
:0F021E0007EDF452A1ED42A2BB0203ED42A12273
:1003CB00EF70028D80BF01028D90BF02028DA022C3
:10039300EF7003ED4280BF0103ED4290BF0203ED16
:0303A30042A02253
:10032800EF7004EDF45280BF0104EDF45290BF0267
:0603380004EDF452A022C6
:0F03DB00EF7003AF8022BF0103AF9022AFA022CB
:10036A00EF7005E5805DFF22BF0105E5905DFF2284
:05037A00E5A05DFF227B
:1003A600538F1FE4F59DF59EF595F59F53A9FE53D2
:0303B600B9FE226B
:08042400E58F54DF4FF58F2234
:1002D900E58F543F4440F58FE59E54FA4F4517F595
:0E02E9009EE59D54804D4B45154516F59D2212
:0B03F800EF6004439D8022539D7F2294
:03042C008F9F227D
:03042F00AF9F225A
:0E03EA00E58F543F4480F58FEF54FEF59E22C0
:0B040300EF6004439D0822539DF72288
:0B040E00EF6004439E0122539EFE227B
:0B041900EF6004439D8022539D7F2272
:030432008F9F2277
:03043500AF9F2254
:10022D008F0B8E0A8D098C08438FC0E59D540F45A9
:10023D00104511F59DAB0FAA0EA90DA80CAF0BAE75
:10024D000AAD09AC0812013CE4FB7A01F9F8120180
:10025D003C8F95AB0FAA0EA90DA80CAF0BAE0AAD36
:09026D0009AC0812013C8F9E222D
:030438008F9F2271
:03043B00AF9F224E
:0403B900AD07AC06DA
:0D03BD00EC6005439D088003539DF78D9F64
:0103CA002210
:10033E00E59D540475F040A4AD9F7C002DFFEC3577
:05034E00F0FE539DFBD1
:010353002287
:10035400EF600543A901800353A9FEED600443B98E
:06036400012253B9FE2244
:1002B100EF64806008EF64406003BF080DE59E5F56
:1002C10060047E01800FE4FE800BE59D5F60047E8B
:0702D100018002E4FEAF060C
:0102D8002203
:10031100EF64806008EF64406003BF0805EFF452AA
:070321009E22EFF4529D2221
:030000000202F702
:1002F70078FFE4F6D8FD9000007F007E01E4F0A3CC
:0A030700DFFCDEFA758117020276B2
:1001000075F008758200EF2FFFEE33FECD33CDCCB6
:1001100033CCC58233C5829BED9AEC99E582984039
:100120000CF582EE9BFEED9AFDEC99FC0FD5F0D616
:10013000E4CEFBE4CDFAE4CCF9A88222B800C1B940
:100140000059BA002DEC8BF084CFCECDFCE5F0CB7E
:10015000F97818EF2FFFEE33FEED33FDEC33FCEBB7
:1001600033FB10D703994004EB99FB0FD8E5E4F972
:10017000FA227818EF2FFFEE33FEED33FDEC33FC5F
:10018000C933C910D7059BE99A4007EC9BFCE99A53
:10019000F90FD8E0E4C9FAE4CCFB2275F010EF2F98
:1001A000FFEE33FEED33FDCC33CCC833C810D70798
:1001B0009BEC9AE899400AED9BFDEC9AFCE899F8D3
:0E01C0000FD5F0DAE4CDFBE4CCFAE4C8F92266
:00000001FF
